:102F000010E0A0E6B0E0E0ECF3E302C005900D9223
:102F1000AA36B107D9F711E0AAE6B0E001C01D92C8
:102F2000A03AB107E1F7112492C0089582E390E03E
:102F3000089515BA8BEB87BBC09814BA82E081BBA9
:102F40008BE085BD85EE83BD88E083BF8FEF8CBFAE
:102F50000895FF920F931F93CF93DF931091710009
:102F60001C5FF09072008DE18093700010927100F0
:102F7000C0E0D0E00BC0FF27E059FF4F80810E94E6
:102F80003B19E02FFF27E059FF4F8083EC2FEC5FC8
:102F90000C2F0E5F21969E012D5F211760F3EF2D00
:102FA000FF27E059FF4F1282E5E0CDB7DEB70C9462
:102FB000BE19809172000E943B19982F8091710078
:102FC000813011F490937200809173000E943B193C
:102FD000982F80917100823011F49093720080914B
:102FE00074000E943B19982F80917100833011F476
:102FF00090937200809175000E943B19982F8091E8
:103000007100843011F4909372000895EF92FF9252
:103010000F931F93CF93DF938C010E94CB188EE008
:103020000E94B418C0E0D0E080E7E82E80E0F82EDF
:1030300006C0F70181917F010E94B4182196C01744
:10304000D107B9F7E6E0CDB7DEB70C94BD19A0E023
:10305000B0E0EDE2F8E10C949E190E9499170E94ED
:10306000A6180E94FD18A0E0B0E00E94CC19802DA7
:1030700080939C01789483B7887E83BFC398CC24C7
:10308000DD24BB24EE24FF2400E004C00BE1C1E0FA
:10309000D0EF02C0C0E0D0EF0E94AC182FEF8F3FFE
:1030A0009207D1F3182F20EFC030D20719F48B31DB
:1030B00099F7ECCF20EFC130D20729F40827B82EBA
:1030C000C2E0D0EFE9CF20EFC230D20739F4992720
:1030D000F82EEE240127C3E0D0EFDECF20EFC3307F
:1030E000D20739F49927E82AF92A0127C4E0D0EF5A
:1030F000D3CF20EFC430D20741F48E3059F60827E1
:10310000CC24DD24C5E0D0EFC7CF20EFC530D207F7
:1031100081F4F601E059FF4F80830894C11CD11C53
:103120000827CE14DF0409F0B7CF7601C6E0D0EF50
:10313000B3CF80EFC630D80709F0AECF101709F033
:10314000A9CF8B2D0E94021A012FA4CF88E18AB942
:1031500083E089B910BC08955F9903C08FEF9FEF9A
:1031600008958CB199270895982F5D9BFECF9CB947
:1031700080919E01892780939E010895CF93DF93CC
:10318000EC0103C00E94B418219688818823D1F7EE
:10319000DF91CF9108950F931F938C01812F992771
:1031A0000E94B418802F0E94B4181F910F910895A7
:1031B00010929E01089580919E010E94B418109271
:1031C0009E01089588B788B78F7B88BF10929F01B2
:1031D00081E090E008959C018BE085BD08C088B730
:1031E00088B78F7B88BF10929F01215030402115F6
:1031F0003105A9F715BC14BC08951DB887B38F75A8
:1032000087BBC19AB89A089590919C01933021F49C
:1032100084E080939C010895923021F41EB883E5E8
:103220008DB90895892F8E7F21F4709A91709F5ADD
:103230009DB9089590919C0180E013C000000000AA
:10324000000000000000000000000000000000007E
:10325000000000000000000000000000000000006E
:103260008F5F891759F70895C79A0E941A19C7984E
:103270000E941A190895FF920F931F93182F80919F
:103280009C01833030F41FB9779BFECF8FB1992713
:1032900011C0FF24C59817FDC59A000FB6990160AB
:1032A0000E943419F39488E0F81611F0110FF2CF50
:1032B000802F99271F910F91FF9008950F931F93CF
:1032C0008C01812F99270E943B19802F0E943B1966
:1032D00099271F910F910895EF92FF920F931F93DB
:1032E0007B018C01892F9927AA27BB270E943B19B4
:1032F000C801AA27BB270E943B19BB27A12F902FEB
:103300008F2D0E943B198E2D0E943B1999271F91EA
:103310000F91FF90EF900895C19AB89A82E090E0E3
:103320000E94EB18B898C19808952F923F924F923F
:103330005F926F927F928F929F92AF92BF92CF9245
:10334000DF92EF92FF920F931F93CF93DF93CDB74E
:10335000DEB7CA1BDB0B0FB6F894DEBF0FBECDBFC6
:1033600009942A88398848885F846E847D848C8497
:103370009B84AA84B984C884DF80EE80FD800C81A0
:103380001B81AA81B981CE0FD11D0FB6F894DEBF83
:103390000FBECDBFED010895E199FECFBFBBAEBB1F
:1033A000E09A11960DB20895E199FECFBFBBAEBB76
:1033B0000DBA11960FB6F894E29AE19A0FBE0895ED
:0A33C0004156524953505F3200009D
:043400000C94801791
:10340400A0E0B0E0E8E0FAE10C949619382E409080
:103414006B0050906C0060906D0070906E00109185
:103424007000113081F41092710088E08093720072
:10343400A3E7B0E0E0E6F0E001900D928150E1F7FF
:10344400CBE0D0E05BC4123021F5809171008E395D
:10345400A9F08F39C1F08839D1F49091720090931A
:103464009C0120E030E0D9010E94CC19802D9817EE
:1034740071F0D901092E0E94D41909C080917200FB
:1034840080936A0004C08091720080936F0082E090
:10349400B3C3133051F580917100823971F08339CF
:1034A40028F4803971F0813951F40DC08E3981F0DE
:1034B4008F3989F0883919F408C09AE00EC090E079
:1034C4000CC09DE10AC092E008C090919C0105C027
:1034D40090916A0002C090916F0083E08093700025
:1034E4001092710090937200E6C31630D1F52091CA
:1034F4007100332744275527522F44273327222787
:10350400809172009927AA27BB27DC019927882775
:10351400282B392B4A2B5B2B809173009927AA27E0
:10352400BB27BA2FA92F982F8827282B392B4A2B52
:103534005B2B809174009927AA27BB27282B392B52
:103544004A2B5B2B20936B0030936C0040936D00EF
:1035540050936E001093700010927100C2E0D0E09E
:10356400CDC3103109F068C081E080939D010E94B1
:10357400931E8091720099270E94EB18C39883B719
:10358400856183BFC0E0D0E045C0809178000E948F
:103594003B198091750099270E94EB18809179005E
:1035A4000E943B198091750099270E94EB18809125
:1035B4007700833079F480917A000E943B19182FA8
:1035C4008091750099270E94EB1880917B000E94DE
:1035D4003B190EC080917A000E943B1980917500BE
:1035E40099270E94EB1880917B000E943B19182FA9
:1035F4008091750099270E94EB1880917600181726
:1036040009F488C380917700882309F483C30E9456
:1036140034192196809174009927C817D90708F4A2
:10362400B4CF80E180937000CF3FD10509F494CFEB
:1036340080EC8093710092CF113149F410929D0176
:103644000E94FD1883B7887E83BFC39883CF12314D
:1036540021F5809173000E943B19809174000E94AF
:103664003B19809175000E943B19809176000E945D
:103674003B1980917200882331F48091710099275D
:103684000E94EB1808C060E070E080E090EF0E94B8
:103694006C1980FDF8CF82E1AFC2133109F03DC14E
:1036A400809171009927982E88248091720099271F
:1036B400882A992AD0907300D0FE08C0AA24BB247B
:1036C400EE24FF248701CAE7D0E0D7C0AA24BB2494
:1036D400EE24FF248701CAE7D0E079C0C5018170D8
:1036E4009070C82E882321F080917500886002C0F4
:1036F400809175000E943B1980916B0090916C0041
:103704000E945E1988810E943B19909178008881FB
:10371400981789F0E0906B00F0906C0000916D00B8
:1037240010916E008FEF9FEFA0E0B0E0E822F92245
:103734000A231B2304C091EFD922A2E0DA2A8D2D9B
:1037440099278E7090708230910519F1843091051B
:10375400A9F4CC2021F080917700886002C0809188
:1037640077000E943B19C7010E945E1980E00E9405
:103774003B1990917800891789F4EBCF089749F4A5
:1037840060E070E080E090EF0E946C1980FF06C05A
:10379400F7CF8091740099270E94EB18CC2099F000
:1037A40080916B0090916C00A0916D00B0916E00BF
:1037B4000196A11DB11D80936B0090936C00A093A2
:1037C4006D00B0936E000894A11CB11C2196A8143E
:1037D400B90409F083CF9FC0C50181709070C82ED1
:1037E400882321F080917500886002C08091750063
:1037F4000E943B1980916B0090916C000E945E19AD
:1038040088810E943B199091780088819817E1F093
:10381400E0906B00F0906C0000916D0010916E00D0
:103824008FEF9FEFA0E0B0E0E822F9220A231B23E8
:10383400EE0CFF1C001F111FCC20D9F00894E11CD2
:10384400F11C011D111D02C0CC2099F080916B0068
:1038540090916C00A0916D00B0916E000196A11D35
:10386400B11D80936B0090936C00A0936D00B09396
:103874006E000894A11CB11C2196A814B90409F087
:10388400ABCFD7FE48C0809176000E943B19C2019D
:103894000E945E1980E00E943B19E114F1040105C5
:1038A400110521F49FE8D922A0E1DA2A8D2D992768
:1038B400807790708031910549F180329105D1F47F
:1038C400E0FE04C080917700886002C08091770098
:1038D4000E943B19D801C701B695A795979587957E
:1038E4000E945E1980E00E943B199091780089172C
:1038F40091F4E6CF8034910549F460E070E080E013
:1039040090EF0E946C1980FF06C0F7CF809174007D
:1039140099270E94EB1883E16FC1143109F053C059
:10392400809171009927182F0027809172009927A0
:10393400082B192BD0907300EE24FF24C2E7D0E0AB
:1039440035C0E0FE22C08D2D88600E943B19809115
:103954006B0090916C000E945E1980E00E943B19FC
:10396400888380916B0090916C00A0916D00B09160
:103974006E000196A11DB11D80936B0090936C00A5
:10398400A0936D00B0936E000DC08D2D0E943B1965
:1039940080916B0090916C000E945E1980E00E94FF
:1039A4003B1988830894E11CF11C2196E016F1066A
:1039B40041F6E801239684E180937000109271002F
:1039C40000591F4F5DC1153109F019C18091710073
:1039D4009927B82EAA24809172009927A82AB92A77
:1039E400D0907300D0FE06C0EE24FF248701C0E708
:1039F400D0E0B5C0EE24FF248701C0E7D0E06DC05D
:103A0400809175000E943B1980916B0090916C002D
:103A14000E945E198A850E943B199A8580917800DC
:103A24009817A9F080917900981789F0E0906B00BD
:103A3400F0906C0000916D0010916E008FEF9FEF7D
:103A4400A0E0B0E0E822F9220A231B2304C091EF8E
:103A5400D922A2E0DA2A8D2D99278E7090708230B7
:103A6400910511F184309105A1F4809177000E94B1
:103A74003B19C7010E945E1980E00E943B19982FF0
:103A840080917800981789F380917900981769F3E9
:103A940010C0089749F460E070E080E090EF0E9465
:103AA4006C1980FF06C0F7CF8091740099270E949B
:103AB400EB1880916B0090916C00A0916D00B09117
:103AC4006E000196A11DB11D80936B0090936C0054
:103AD400A0936D00B0936E002196C50180599F4F4D
:103AE400C817D90709F08CCF86C0809175000E9451
:103AF4003B1980916B0090916C000E945E198A853D
:103B04000E943B199A85809178009817A1F08091C2
:103B14007900981781F0E0906B00F0906C000091B0
:103B24006D0010916E008FEF9FEFA0E0B0E0E822EF
:103B3400F9220A231B2380916B0090916C00A091C1
:103B44006D00B0916E000196A11DB11D80936B00B4
:103B540090936C00A0936D00B0936E002196C50104
:103B640080599F4FC817D90709F0BFCFD7FE43C06C
:103B7400809176000E943B19C2010E945E1980E088
:103B84000E943B19E114F1040105110521F49FE899
:103B9400D922A0E1DA2A8D2D99278077907080317F
:103BA400910521F180329105A9F4A0FE04C0809111
:103BB4007700886002C0809177000E943B19C7019A
:103BC4000E945E1980E00E943B1990917800891749
:103BD40091F4EBCF8034910549F460E070E080E02B
:103BE40090EF0E946C1980FF06C0F7CF809174009B
:103BF40099270E94EB1885E180937000ADCC1631B3
:103C040009F041C0809171009927D82FCC27809169
:103C140072009927C82BD92BF090730000E710E0AD
:103C240023C08F2D0E943B1980916B0090916C00F2
:103C34000E945E1980E00E943B19F8018283809102
:103C44006B0090916C00A0916D00B0916E00019694
:103C5400A11DB11D80936B0090936C00A0936D0027
:103C6400B0936E000F5F1F4FCE0180599F4F08170E
:103C74001907B9F6239686E18093700010927100BB
:103C8400F801128239C01731C9F4809171000E9481
:103C94003B19809172000E943B19809173000E942D
:103CA4003B19809174000E943B191093700010928C
:103CB400710010927200C3E0D0E020C0183141F0CE
:103CC400193119F31A3121F01B3111F01C3159F457
:103CD4000E94D91710937000109271001092730013
:103CE400C4E0D0E00BC01D31B9F480917200C82F3C
:103CF400DD2723960E94A917209771F08BE10E947B
:103D0400B418832D0E94B418CE010E9406180E9494
:103D1400DB1802C080E170CFE1E1CDB7DEB70C94CF
:023D2400B219D2
:103D2600B898C19882E090E00E94EB1888B38F752E
:103D360088BB87B3806A87BBC19AB89A80E00000C7
:103D46008F5F883CE1F7B898C19882E090E00E94C6
:083D5600EB180E940419089506
:0400000300002F00CA
:00000001FF
